:1000000075815053877F538930438920758DFDD288
:100010008E759840D29CC2981200D112010802003D
:1000200021C298D2B23098FDC2B2C298E599B441CB
:10003000091200D112008302007FB442091200D1DC
:1000400012009002007FB443091200D112009D02F9
:10005000007FB444091200D11200AA02007FB44507
:10006000061200D102007FB446091200D11200B777
:1000700002007FB447091200D11200C402007FC2FF
:100080009880A0C294D295D292C293D290D291225B
:10009000D294C295C292D293D290D29122C294C2EB
:1000A00095D292C293D290D29122C294D295C2920A
:1000B000C293D290D29122C294D295C292D293D2BC
:1000C00090D29122D294C295D292C293D290D291E0
:1000D00022C290C291C294C295C292C29322697008
:1000E00063637A7173706B666475742F64706E7578
:1000F0000930D509FD22750A0A11EFD50AFB2275D0
:100100000C0A11F6D50CFB227C0A11FFDCFC223113
:10011000083108310831083108227C6411FFDCFC09
:0101200022BC
:00000001FF
